:1018DA004346442D393530000218FD00002B312EC5
:1018EA0030560000000100000218FD00002B322EC5
:1018FA0035560000000100020218FD00002B332EAD
:10190A0033560000000100040218FD00002D352E98
:10191A0030560000000100060218FD0000566F6CE8
:10192A0074616765340100080218FD0000566F6C87
:10193A00746167653501000A0218FD0000566F6C74
:10194A00746167653601000C0218FD000057616C6E
:10195A006B0000000001000E0134000000425554E3
:10196A00544F4E000001001001340000004348416A
:10197A004E4E454C0001001101340000004D4F4409
:10198A0045000000000100120218FD0000544852F0
:10199A005F434831000100130218FD000054485209
:1019AA005F434832000100150218FD0000544852F6
:1019BA005F434833000100170218FD0000544852E3
:1019CA005F434834000100190218FD0000544852D0
:1019DA005F4348350001001B0218FD0000544852BD
:1019EA005F4348360001001D0218FD0000544852AA
:1019FA005F4348370001001F0218FD000054485297
:101A0A005F434838000100210218FD000057414C8D
:101A1A004B5F4348310100230218FD000057414C37
:101A2A004B5F4348320100250218FD000057414C24
:101A3A004B5F4348330100270218FD000057414C11
:101A4A004B5F4348340100290218FD000057414CFE
:101A5A004B5F43483501002B0218FD000057414CEB
:101A6A004B5F43483601002D0218FD000057414CD8
:101A7A004B5F43483701002F0218FD000057414CC5
:101A8A004B5F4348380100310218FD0000574944B2
:101A9A0054485F43310100330218FD00005749449E
:101AAA0054485F43320100350218FD00005749448B
:101ABA0054485F43330100370218FD000057494478
:101ACA0054485F43340100390218FD000057494465
:101ADA0054485F433501003B0218FD000057494452
:101AEA0054485F433601003D0218FD00005749443F
:101AFA0054485F433701003F0218FD00005749442C
:101B0A0054485F4338010041013400000044454C09
:101B1A0041595F4331010043013400000044454C00
:101B2A0041595F4332010044013400000044454CEE
:101B3A0041595F4333010045013400000044454CDC
:101B4A0041595F4334010046013400000044454CCA
:101B5A0041595F4335010047013400000044454CB8
:101B6A0041595F4336010048013400000044454CA6
:101B7A0041595F4337010049013400000044454C94
:101B8A0041595F433801004A023400000057414C72
:101B9A004B5F415F4D01004B02340000005749443E
:101BAA0054485F425501004D00000000000000004B
:081BBA00000000000000000023
:102DC200011F010360FF18E2015700015C00015D71
:042DD20000015E009E
:021E5C008F3CB9
:101E5E00E4F5BA75BCE075E88075D10375D480756C
:101E6E00D78075A57FD293C294C296D2977FD07E2B
:101E7E0007122CE5122CBA7B027D017F507E0012D8
:101E8E002CC27B017D017F537E00122CC2E4FB7DB0
:101E9E00017F49FE122CC27FF47E01122CE5122C1A
:101EAE00BA7B027D017F437E00122CC27B017D0135
:101EBE007F467E00122CC2E4FB7D017F44FE122C75
:101ECE00C27FF47E01122CE5122CBA7B027D017FBB
:101EDE00397E00122CC27B017D017F357E00122CD3
:101EEE00C2E4FB7D017F30FE122CC27FF47E011214
:101EFE002CE57F56122CBC7B027D017F317E0012B9
:101F0E002CC27B017D017F2E7E00122CC2E4FB7D54
:101F1E00017F30FE122CC2754501E5455407F59040
:101F2E00E4F53CE53C25E02413F582E43400F5832A
:101F3E00E0FEA3E07802C333CE33CED8F912284A9E
:101F4E0012000EC293053CE53CC3940840D575457E
:101F5E0002E5455407F590E4F53CE53C25E02423E5
:101F6E00F582E43400F583E0FEA3E07802C333CEBD
:101F7E0033CED8F912284A12000EC293053CE53C26
:101F8E00C3940840D5754504E5455407F590E4F52E
:101F9E003CE53C25E02433F582E43400F583E0FE95
:101FAE00A3E07802C333CE33CED8F912284A1200FA
:101FBE000EC293053CE53CC3940840D5754503E538
:101FCE00455407F59090004BE0FEA3E0FF12286DFC
:101FDE0012000EC293754505E5455407F590900025
:101FEE004DE0FEA3E0FF12286D12000EC293754560
:101FFE0006E5455407F590E4F544F543F542F54101
:10200E00F53CAF44AE43AD42AC4178041212D28FD0
:10201E00448E438D428C417443253CF582E434005A
:10202E00F583E0FFEF4544F544E543F543E542F51E
:10203E0042E541F541053CE53CB408C6AF44AE432C
:10204E00AD42AC41122A5612000EC293754501E5FF
:05205E00455407F59058
:01206300225A
:092E3300151EA81EEFF6051E2273
:052E42008F327F002229
:102C8D008B328A338934121055AB35AA36A93712D7
:102C9D00109BAB32AA33A93490000112106EAB35E4
:0D2CAD00AA36A9379000011210AD7F022257
:1023D600E55C7017E557045407F557540FF5BB75C0
:1023E600BCE0E4F55BF55AF559F558E4F538C2AFAB
:1023F600C2EDD2EC30EDFDD2AFAFBFEFFEADBEED1C
:10240600FFE4FCFDE55B2FF55BE55A3EF55AED353D
:1024160059F559EC3558F5581229250538E538C3CC
:10242600941040CA055CE55C704AAF5BAE5AAD5984
:10243600AC58FB7A01F9F81212218F5B8E5A8D592E
:102446008C58E4120F96E4FBFA79807847120EF95D
:102456007B007A40791C7845120DF0C2AF120FD47A
:10246600E55725E02400F582E43400F583EEF0A379
:04247600EFF0D2AF02
:01247A00223F
:10284A00F53E8E3D533EFC533D0FE53C754000C4BA
:10285A0054F0F53FE540253EF53EE53F353DF53D73
:03286A00AF3EFE80
:04286D008E508F51A9
:10287100D293E4F552E47E80A852088005CEC313BA
:10288100CE13D8F9FFE5505EFEE5515F4E7003D3DC
:102891008001C392967F0A7E00122B0ED2947F0A8A
:1028A1007E00122B0EC2947F0A7E00122B0E05525F
:0728B100E552C3941040BE84
:0128B80022FD
:082A56008F4A8E498D488C4720
:102A5E00D293E4F54BE47F01FEFDFCA94BC8E9C817
:102A6E001212D2EF554AFFEE5549FEED5548FDECD8
:102A7E005547FCE4FBFAF9F8C31212C17003D38078
:102A8E0001C392967F0A7E00122B0ED2947F0A7E8D
:102A9E0000122B0EC2947F0A7E00122B0E054BE500
:062AAE004BC3942040AF71
:012AB40022FF
:10000E00D2957F0A7E00122B0EC2957F0A7E0002C9
:02001E002B0EA7
:0926D300F583E0FEA3E0FFAD5E1B
:0626DC008E478F488D4976
:1026E20085494A754907E5495407F590754E0375C2
:1026F2004FE8E4F54DAC4EAD4FAE47AF481210E196
:102702008E4B8F4CAE47AF48AC4EAD4F1210E18CA2
:10271200478D48AE4EAF4F7C007D0A1210E18E4EBF
:102722008F4FC37403954DFFEFFEE54C2430FDE45B
:10273200354B4EFEEDFF12286D12000EC293054D71
:10274200E54DC3940440AE854A49E5495407F590E6
:012752002264
:082CBA007F207B037D017E00F9
:102CC2008D477D07ED5407F590CDEFCDCCEECCEBE3
:102CD2004CFEEDFF12286D12000EC293E547540719
:022CE200F5906B
:012CE40022CD
:10074B00E4F544F543F542F54185803853383C9048
:10075B000010E538F0643C7003020DEFE538641CC3
:10076B00702CE55D045407F55D855E3AE4F55EE5B6
:10077B005E5407F590AF5D7E0012286DC293853AEB
:10078B005EE55E5407F5907F2C7E01122CE5900000
:10079B0011E55DF0E538B42C11E55E0475F00784C6
:1007AB0085F05E7F2C7E01122CE5900012E55EF049
:1007BB005407F590E55EB407004003020DEF900778
:1007CB00D0F82828730207E502087A02096F020A9B
:1007DB0064020B2B020C20020CED7B037D017F507E
:1007EB007E00122CC27B027D017F527E00122CC236
:1007FB007B017D017F4F7E00122CC2E4FB7D017FCC
:10080B004DFE122CC2E53864346003020DEF78966E
:10081B0076F112247B7B037D017F737E00122CC249
:10082B007B027D017F617E00122CC27B017D017FEB
:10083B00767E00122CC2E4FB7D017F65FE122CC27A
:10084B007FF47E01122CE5122CBA7B027D017F20F6
:10085B007E00122CC27B017D017F6F7E00122CC2A9
:10086B00E4FB7D017F6BFE122CC27FF4020DEAE5E7
:10087B003864347044E55D25E02413F582E43400DC
:10088B00F583E475F00112116CE55D25E02413F599
:10089B0082E43400F583E0FEA3E07003EE640470A1
:1008AB0011E55D25E02413F582E43400F583E4F0D3
:1008BB00A3F07F647E00122CE5E53864387042E5C6
:1008CB005D25E02413F582E43400F583E0FEA3E01C
:1008DB004E7013E55D25E02413F582E43400F583B7
:1008EB007404F0A3E4F0E55D25E02413F582E43411
:1008FB0000F58374FFF5F012116C7F647E00122CEF
:10090B00E5E55D25E02413F582E434001226D3E5FA
:10091B005EB4013AE55D25E02413F582E43400F57D
:10092B0083E0FEA3E07802C333CE33CED8F9F53C97
:10093B008E3B533CFC533B0FE55D754600C454F0B6
:10094B00F545E546253CF53CE545353BF53BE538BE
:10095B0064346009E53864386003020DEFAF3CAED8
:10096B003B020CE4E53864347044E55D25E0242358
:10097B00F582E43400F583E475F00112116CE55D4A
:10098B0025E02423F582E43400F583E0FEA3E07038
:10099B0003EE64047011E55D25E02423F582E43455
:1009AB0000F583E4F0A3F07F647E00122CE5E538BC
:1009BB0064387042E55D25E02423F582E43400F5CC
:1009CB0083E0FEA3E04E7013E55D25E02423F58262
:1009DB00E43400F5837404F0A3E4F0E55D25E02432
:1009EB0023F582E43400F58374FFF5F012116C7F6C
:1009FB00647E00122CE5E55D25E02423F582E434CA
:100A0B00001226D3E55EB4023AE55D25E02423F51A
:100A1B0082E43400F583E0FEA3E07802C333CE33E7
:100A2B00CED8F9F53E8E3D533EFC533D0FE55D753B
:100A3B004600C454F0F545E546253EF53EE5453503
:100A4B003DF53DE53864346009E5386438600302F0
:100A5B000DEFAF3EAE3D020CE4E538B4340EE4903E
:100A6B00004BF0A3F07FF47E01122CE5E538B4388F
:100A7B000F74FF90004BF0A3F07FF47E01122CE576
:100A8B00D390004CE0940090004BE094005006E5AE
:100A9B00386438702B7B03AD5E7F4D7E00122CC209
:100AAB007B02AD5E7F417E00122CC27B01AD5E7F6F
:100ABB004E7E00122CC2E4FBAD5E7F2EFE122CC2CA
:100ACB0090004BE07002A3E06006E5386434702BB5
:100ADB007B03AD5E7F417E00122CC27B02AD5E7F3D
:100AEB00557E00122CC27B01AD5E7F547E00122C12
:100AFB00C2E4FBAD5E7F4FFE122CC2E55EB4030A6F
:100B0B0090004BE0F53DA3E0F53EE5386434600919
:100B1B00E53864386003020DEFAF3EAE3D020CE4E6
:100B2B00E53864347044E55D25E02433F582E43424
:100B3B0000F583E475F00112116CE55D25E02433BB
:100B4B00F582E43400F583E0FEA3E07003EE640469
:100B5B007011E55D25E02433F582E43400F583E480
:100B6B00F0A3F07F647E00122CE5E5386438704208
:100B7B00E55D25E02433F582E43400F583E0FEA344
:100B8B00E04E7013E55D25E02433F582E43400F587
:100B9B00837404F0A3E4F0E55D25E02433F582E4EF
:100BAB003400F58374FFF5F012116C7F647E001234
:100BBB002CE5E55D25E02433F582E434001226D3E1
:100BCB00E55EB4043AE55D25E02433F582E43400B8
:100BDB00F583E0FEA3E07802C333CE33CED8F9F52C
:100BEB00408E3F5340FC533F0FE55D754600C454A8
:100BFB00F0F545E5462540F540E545353FF53FE544
:100C0B003864346009E53864386003020DEFAF4097
:100C1B00AE3F020CE4E538B4340F74FF90004DF096
:100C2B00A3F07FF47E01122CE5E538B4380EE49086
:100C3B00004DF0A3F07FF47E01122CE5D390004E13
:100C4B00E0940090004DE094005006E53864347059
:100C5B002B7B03AD5E7F427E00122CC27B02AD5E0E
:100C6B007F4C7E00122CC27B01AD5E7F4B7E00124F
:100C7B002CC2E4FBAD5E7F2EFE122CC290004DE029
:100C8B007002A3E06006E5386438702B7B03AD5E21
:100C9B007F557E00122CC27B02AD5E7F507E001210
:100CAB002CC27B01AD5E7F447E00122CC2E4FBADF7
:100CBB005E7F54FE122CC2E55EB4050A90004DE037
:100CCB00F53FA3E0F540E53864346009E538643856
:100CDB006003020DEFAF40AE3F12286D12000EC243
:100CEB009322E538B4342A7443255DF582E434004D
:100CFB00F583E004F07443255DF582E43400F5835D
:100D0B00E0B4100D7443255DF582E43400F583E403
:100D1B00F0E538B4382A7443255DF582E43400F5E8
:100D2B0083E0700E7443255DF582E43400F5837423
:100D3B0010F07443255DF582E43400F583E014F084
:100D4B007443255DF582E43400F583E0FF7E007C7F
:100D5B00007D051210CFEF240AFFE43EFE7D6412E6
:100D6B0010CFAD5E1226DC7B01AD5E7F6E7E001276
:100D7B002CC2E4FBAD5E7F73FE122CC2E55EB406A3
:100D8B0006855D39E4F55DE4FBAF44AE43AD42ACA3
:100D9B004178041212D28F448E438D428C4174439E
:100DAB002BF582E43400F583E0FFEF4544F544E591
:100DBB0043F543E542F542E541F5410BBB08CA85D6
:100DCB00395DE53864346005E538B43817AF44AEA7
:100DDB0043AD42AC41122A5612000EC2937F2C7EB9
:040DEB0001122CE5E0
:010DEF0022E1
:062E3C001223D602074B31
:0D2E0100245265763A203335353820240000
:032DD60001960063
:101BC200E47896F6122DF375E104E4F5E275E3404C
:101BD20075A401F5A5F5A675A72075B16775B208BC
:101BE200122AB5E4FF122DA4E4F53AF53B7D01AFCC
:101BF2003B122D39053BE53B7002053AC39401E5E2
:101C02003A940040E8E4F520C20BC208C20FC20EAB
:101C1200C20D7896F6C2B57874F67872F618F67830
:101C220078F6F53AF53B747A253BF8E4F6053BE5A0
:101C32003B7002053A6414453A70EBE4F53AF53B21
:101C4200748E253BF8E4F6053BE53B7002053A64E9
:101C520008453A70EBE5EF20E10CE5EF5408D39428
:101C6200004003D38001C392037D08E4FF122D607C
:101C7200E47877F6786FF6AB60AA61A962786FE6CE
:101C8200FF75F010A4F58285F08312106EFE78774E
:101C920026F6EE6005786F0680DDEFD394004028CB
:101CA200AB60AA61A96290000D1212F17455121074
:101CB2009B12105564556002D20D74AA12109B1229
:101CC200105564AA6002D20D1222618F39E53920C3
:101CD200E035C20A74FFF508F509F50AF50B7E0036
:101CE2007F107D007B007A00790E121347753FFF4B
:101CF2007540187541DA7542007543107B007A0011
:101D0200790E122BB28002D20A902E08E493FF338E
:101D120095E0FEEF24D0FFEE34FFFE7C007D6412DE
:101D220010CFAA06AB07902E07E493FF3395E0FE8F
:101D3200EF24D0FFEE34FFFE7C037DE81210CFEFDC
:101D42002BFBEE3AFA902E09E493FF3395E0FEEF77
:101D520024D0FFEE34FFFE7C007D0A1210CFEF2B61
:101D6200FFEE3AFEA3E493FD3395E0FCED24D0FDB3
:101D7200EC34FFCD2FF50DED3EF50CE53930E103E6
:101D8200021E33E4F53AF53BE53BC4F8540FC8684C
:101D9200FFE53AC454F048FEAB60AA61A9628F82A3
:101DA200F58312106E7003021E2AE92FF9EA3EFA39
:101DB20090000412106E20E264E4F538E538C3782E
:101DC2001F965059E53BC4F8540FC868FFE53AC462
:101DD20054F048AB60AA61A9628F82F58312106E3B
:101DE200FF7E00C006C0077D00E53BC4F8540FC863
:101DF20068FFE53AC454F048FEE92FF9EA3EFA904A
:101E0200000D1212F17877E68538F0A429F9EA3547
:101E1200F0FAD007D0061213470538809F053BE53C
:101E22003B7002053A021D8A7F01121E5CC20C80C1
:101E320007E4FF121E5CD20CE4F53AF53B7A007B14
:101E4200967D03AF3B1227D1053BE53B7002053A75
:091E5200C39401E53A940040E458
:011E5B002264
:052E47007878E6FF228F
:0300230002216E49
:10216E00C0E0C0F0C083C082C0D075D000C000C037
:10217E0001C002C003C004C005C006C00730992FBD
:10218E00C2997872067972E778746670117872F671
:02219E00D20964
:0821A00075230A0000D523FBA2
:0421A800C2B580112B
:0821AC007523140000D523FB8C
:1021B4007872E6248EF8E6F59920980302224620E8
:1021C4009A07200B04C2988075C29A7871E6062497
:1021D4007AF8A699C2987871E6FFB40113787AE682
:1021E400FE70057871F6805AEE540724027879F669
:1021F400EFB4020E7879E6B40908787BE624037913
:1022040079F77871E6FFB4140476008035EFC3786B
:102214007996402E7871E624FFFDE434FFFC7B00C0
:102224007A00797A1225BB7871E62479F8E66F6032
:0322340002800B1A
:082237007523140000D523FB00
:10223F0012002678717600D007D006D005D004D0D2
:10224F0003D002D001D000D0D0D082D083D0F0D034
:02225F00E0326B
:1028B900787BE675F010A4AB602562F9E56135F027
:1028C900FA90000D1212F17878E6FF18E68FF0A45D
:1028D9002526F582E435F0F58312106EFF7B007A28
:0328E9000079244F
:1028EC008F328B338A348935EA494B601612105576
:1028FC00FFE532FD7C00120003AB33AA34A935EF9F
:03290C0012109B0B
:08290F007536140000D536FBFB
:0E2917008532997F01122D103099FDC2992250
:082DDD007874EFF6C209D2B5CB
:082DE5007532140000D532FB29
:062DED00788EE6F5992244
:102C0400C9EFC9E964017028EDC39B4034781FE61D
:102C1400FFEB2FFFE433FEEDC39FEE6480F8748076
:102C240098501ED20BC3ED9B7878F6787376012208
:102C3400B90214ED6B700AD20B7878F678737602C9
:082C440022C20BE47873F622B2
:1029F500C9EFC9BAFF15BBFF12ED6B7002EC6A7027
:102A050049D20B7878F67873E9F622E964017025E6
:102A1500C3ED9BEC9A401C781FE62BFFE43AFEC3FE
:102A2500ED9FEC9E500DD20BC3ED9B7878F6787335
:102A35007601228015B90218ED6B7002EC6A700AF6
:102A4500D20B7878F67873760222C20BE47873F6A7
:012A5500225E
:10002600787AE6FF54F8F525EF121321006F0900E0
:100036007A0A00891000921100A11200B41900C8B2
:100046001A00E72000ED2801872902853302B4371C
:1000560002D73902F04102F9490302500346610210
:100066004B70033E9800000371787BE6FDE509FBC3
:100076007F018021787BE6FC08E6FDAB09AA087FB4
:10008600018025D20B78737603020371787BE6FD37
:10009600E50BFB7F02122C04020371787BE6FC0859
:1000A600E6FDAB0BAA0A7F021229F5020371787BE3
:1000B600E6FDE509FB7F01122C04200B0302037108
:1000C6008016787BE6FC08E6FDAB09AA087F0112DC
:1000D60029F5200B03020371788E76787F010203DF
:1000E6006E75EF10020371C2ACE4F524D2B5FB7A4B
:1000F6000079247F7F1228EC7B007A0079247F1810
:100106001228EC7B007A0079247F051228EC786FA0
:10011600E61228E57B007A007924AF081228EC7BEA
:10012600007A007924AF091228EC7B007A00792442
:10013600AF0A1228EC7B007A007924AF0B1228EC68
:100146007B007A007924AF0C1228EC7B007A0079C8
:1001560024AF0D1228ECE4F526740E2526F8E612D7
:1001660028E50526E526C3941040EE7B007A007943
:0601760000AF241228EC8A
:08017C0075310A0000D531FBCA
:10018400020238787BE6FFC3786F96400302023F91
:10019400EF75F010A42562F9E56135F085602EF560
:1001A4002F8930C2ACE4F524D2B5FB7A0079247FE0
:1001B4007F1228EC7B007A0079247F0D1228ECABA7
:1001C4002EAA2FA9301210551228E5AB2EAA2FA95A
:1001D400309000011228E2AB2EAA2FA93090000221
:1001E4001228E2AB2EAA2FA9309000031228E2AB0A
:1001F4002EAA2FA9309000041228E2E4F526AB2E93
:10020400E5302405F9E4352FFA7E00E92526F9EED8
:100214003AFA1210551228E50526E526C39408403B
:0C022400DD7B007A007900AF241228EC8A
:0802300075310A0000D531FB15
:10023800C2B5D2AC020371788E7678E408F67F02F4
:1002480002036E122E1B78971212E5788E767C7850
:1002580097E6788FF67898E67890F67899E6789128
:10026800F6789AE67892F67C007D057B007A00792C
:100278008E1225BB7893EFF67F0602036E787BE635
:10028800FFB4010B08E6F50808E6F50902033EEF9E
:10029800B40208787CE6F50802033E787BE6B403EE
:1002A8000808E6F50A08E6F50B02033EE4F526E53C
:1002B80026C3787B965016747C2526F8E6FF740EC4
:1002C8002526F8C6EFC60526E526B410E280677A2B
:1002D800007B327D017878E6FF1227D1787BE6FD36
:1002E800E4FF122D60020371787BE624FF920280FE
:1002F80078787BE624FF9201806F7878E660057550
:100308002802800B200E05752803800375280178C4
:100318008E767908A6287C007D027B007A00798E8B
:100328001225BB7890EFF67F03122DDDE5286401D6
:100338007037D20F8002D208789676F1802B7A0037
:100348007B327D017F001227D1788E7679787BE623
:10035800788FF67C007D027B007A00798E1225BBAF
:100368007890EFF67F03122DDDE52564A060030287
:100378000563787AE664A16003020463797BE7C3C6
:10038800786F96400302045AAB60AA61A962787B31
:10039800E6FF75F010A4F58285F08312106EF5283B
:1003A800EF75F010A429F9EA35F0FA90000412105C
:1003B8006E30E230787BE6FF122E428F28788E76F8
:1003C8007F08A628E5282402FDE433FC7B007A0098
:1003D800798E1225BB74902528F8EFF6E5282403BA
:1003E800FF020560787BE6FF122E42C2ACE4F524DA
:1003F800D2B5E528D39406402B7B007A0079247F78
:100408007F1228EC7B007A007924AF281228ECE4CC
:10041800F526E526C3952850071228B9052680F247
:1004280005288018E52824781228E5E4F526E5262D
:10043800C3952850071228B9052680F27B007A0058
:070448007900AF241228EC3B
:08044F0075310A0000D531FBF4
:10045700020554788E76787F01020560787AE66423
:10046700A26003020563786FE6FF787BE6FEC39F11
:10047700400302055A08E6FDC39F400302055AEEF2
:100487009D400302055A18E6F526E4F52CF52DE5FF
:1004970026D3787C965026AF26122E42AB60AA61EF
:1004A700A96275F010E526A4F58285F08312106E17
:1004B700252DF52DE4352CF52C052680D2C2ACE48C
:1004C700F524D2B5FB7A0079247F7F1228ECC3E5A7
:1004D7002D9480E52C940050028007E52C4480126F
:1004E70028E5AF2D1228E6787BE6F526E526D378B2
:1004F7007C965046E4F527AB60AA61A96275F010B7
:10050700E526A4F58285F08312106EFFE527C39FC9
:100517005024E52675F010A429F9EA35F0FA900081
:100527000D1212F17878E6FF18E68FF0A42527124E
:1005370028DB052780C1052680B27B007A00790079
:05054700AF241228ECB6
:08054C0075310A0000D531FBF6
:10055400C2B5D2AC8009788E76787F01122DDDE5A4
:100564002564587047FA7B327D017878E6FF1227BC
:10057400D175350075360075378F7B007A00797B2D
:10058400122C8D8F28E5282478788EF6E52824010E
:10059400FDE433FC7B007A00798E1225BB748F2531
:1005A40028F8EFF6E5282402FF122DDDE525648006
:1005B4006009E5256488600302074A7873E6B4019C
:1005C4000F7A007B327D017878E6FF1227D1801AFA
:1005D400E4F526E526C3781F96500F7A007B327D1A
:1005E40001AF261227D1052680E9787AE65407F56B
:1005F40028B4070A75270108E6F528088005E4F5FC
:1006040027787BE6F5291528E529C3786F964003FA
:10061400020728AB60AA61A96275F010E529A4F568
:100624008285F08312106EFFE528D39F40028F2845
:100634007873E6B401097878E6F52BF52A8009E4A5
:10064400F52A781FE614F52B7878A62A7878E6D36D
:10065400952B400302071CE4F526E526C3952840A4
:1006640003020711E52975F010A4AB602562F9E5D2
:100674006135F0FA90000412106E30E20302070CA8
:1006840090000112106E64387031E528D394044050
:100694000BE5272526247CF8E6FD804E7871E6C319
:1006A4009526FF74782FF8E6FDE52975F010A4ABC4
:1006B400602562F9E56135F0FA802FAB60AA61A983
:1006C4006275F010E529A4F58285F08312106EFF9F
:1006D400C37871E69F252625272479F8E6FDE529C8
:1006E40075F010A429F9EA35F0FA90000D1212F110
:1006F4007878E6FF18E68FF0A4FFE5262FF582E46C
:1007040035F0F583ED1210AD052602065EAF291211
:100714002E337878060206507878A62AE525648870
:100724007024800FE529B4FF1D787CE6F520E525CB
:10073400B48813788E76787871E62479F8E6788F21
:06074400F67F02122DDD1C
:01074A00228C
:10139A007896E664F160030218D9E4F53EF53F2039
:0213AA00091A1E
:0813AC0075440A0000D544FB62
:1013B400053FE53F7002053E64107004E53E642776
:1013C40070E3C2AF75FFDE75FFADE4F53AF5392081
:1013D4009829E4F53EF53F20981DC3E53F9488E540
:0513E4003E94135012BD
:0813E90075440A0000D544FB25
:1013F100053FE53F70E4053E80E0B2B480D48599B5
:1014010039C298E539641A60030214B8F53EF53F14
:0E14110020981DC3E53F9488E53E94135012C9
:08141F0075440A0000D544FBEE
:10142700053FE53F70E4053E80E030989F85993A97
:10143700C298E4F53EF53F20981DC3E53F9488E543
:051447003E9413501259
:08144C0075440A0000D544FBC1
:10145400053FE53F70E4053E80E02098030213D386
:1014640085993AC298E4F53EF53F20981DC3E53FBF
:081474009488E53E9413501228
:08147C0075440A0000D544FB91
:10148400053FE53F70E4053E80E02098030213D356
:0914940085993AC298D2B5C299BB
:08149D007544140000D544FB66
:0614A5007599783099FDF5
:0814AB0075440A0000D544FB62
:1014B300C2B50218CBE5396450706EF53EF53F2096
:0D14C300981DC3E53F9488E53E9413501238
:0814D00075440A0000D544FB3D
:1014D800053FE53F70E4053E80E02098030213D302
:0914E80085993AC298D2B5C29967
:0814F1007544140000D544FB12
:0814F9007599793099FDC29943
:081501007544140000D544FB01
:081509007599013099FDC299AA
:081511007544140000D544FBF1
:06151900E4F5993099FD94
:08151F0075440A0000D544FBED
:0F152700C2B50218CBE5396401702FD2B5C29955
:081536007544140000D544FBCC
:08153E007599783099FDC299FE
:081546007544140000D544FBBC
:06154E00E4F5993099FD5F
:0815540075440A0000D544FBB8
:10155C00C2B50218CBE5396402600302160BF53EE6
:10156C00F53F20981DC3E53F9488E53E9413501237
:08157C0075440A0000D544FB90
:10158400053FE53F70E4053E80E02098030213D355
:1015940085993AC298E4F53BE53A13B392B4E53A37
:1015A40025E0FEC3E4949AEE94135029E53A7F00B3
:1015B40025E0FEC39460501DE5B654F04408F5B62A
:1015C400758F038E408F418541828E83E4F053B63C
:0C15D400F0F58F8003753BFFD2B5C29983
:0815E0007544140000D544FB22
:0815E8007599783099FDC29954
:0815F0007544140000D544FB12
:0615F800853B993099FDCE
:0815FE0075440A0000D544FB0E
:10160600C2B50218CBE53964036003021734F53E10
:10161600F53F20981DC3E53F9488E53E941350128C
:0816260075440A0000D544FBE5
:10162E00053FE53F70E4053E80E02098030213D3AA
:10163E0085993AC298E4F53EF53F20981DC3E53FE3
:08164E009488E53E941350124C
:0816560075440A0000D544FBB5
:10165E00053FE53F70E4053E80E02098030213D37A
:10166E0085993CC298E53A1392B4E53A25E0FEC35B
:10167E00E4949AEE941340030213D3E53A7D0025C9
:10168E00E0FCC3946040030213D3E5B654F0440863
:10169E00F5B6758F01E53C75F020A42DFFE5F03C05
:1016AE00F5408F41E4F53DE53DC394205043E4F50C
:1016BE003EF53F20981DC3E53F9488E53E941350B8
:0116CE001209
:0816CF0075440A0000D544FB3C
:1016D700053FE53F70E4053E80E02098030213D301
:1016E7000541E541AE407002054014F5828E83E561
:1016F70099F0C298053D80B653B6F0E4F58FD2B5A0
:02170700C29985
:081709007544140000D544FBF7
:081711007599783099FDC29929
:081719007544140000D544FBE7
:06172100E4F5993099FD8A
:0817270075440A0000D544FBE3
:10172F00C2B50218CBE539640460030217D0F53E49
:10173F00F53F20981DC3E53F9488E53E9413501262
:08174F0075440A0000D544FBBB
:10175700053FE53F70E4053E80E02098030213D380
:1017670085993AC298E53A25E0F542754300E4F5D4
:101777003BF53EF53F0543E543AE42700205421493
:10178700F5828E83E493253BF53B053FE53F7002E9
:0E179700053E7004E53E640270DBD2B5C299D7
:0817A5007544140000D544FB5B
:0817AD007599783099FDC2998D
:0817B5007544140000D544FB4B
:0617BD00853B993099FD07
:0817C30075440A0000D544FB47
:1017CB00C2B50218CBE539640560030218C3F53EB8
:1017DB00F53F20981DC3E53F9488E53E94135012C6
:0817EB0075440A0000D544FB1F
:1017F300053FE53F70E4053E80E02098030213D3E4
:1018030085993AC298E4F53EF53F20981DC3E53F1C
:081813009488E53E9413501285
:08181B0075440A0000D544FBEE
:10182300053FE53F70E4053E80E02098030213D3B3
:0918330085993CC298D2B5C29916
:08183C007544140000D544FBC3
:0818440075997F3099FDC299EE
:08184C007544140000D544FBB3
:101854007599203099FDE53A25E0FCE53C75F020CA
:10186400A42400FFE5F03CF5428F43E4F53BF53D4D
:02187400C29917
:081876007544140000D544FB89
:10187E00854382854283E493F5993099FD0543E5CE
:10188E0043AE427002054214F5828E83E493253BEB
:0B189E00F53B053DE53DB420CDC299AF
:0818A9007544140000D544FB56
:0618B100853B993099FD12
:0818B70075440A0000D544FB52
:1018BF00C2B58008E539B4060375EF10E539640742
:0A18CF0060030213D37896F6D2AF3F
:0118D90022EC
:102925007F00122D10200A0B7A007B327D017F007B
:102935001227D1300D0B7A007B1E7D017F001227F7
:10294500D1300817300E147A007B327D017878E695
:10295500FF1227D1C20812247BD20A200C0C300E9C
:1029650009789676F112247BD20C300F08300E05CB
:10297500C20F12139A122E0EE47B2C7A01F9F8C3BA
:082985001212C15002D20E2211
:0B2E2800121BC2122925122E3C80F85C
:10206400005EBCE2613FDD83C29C7E20A3FD1F4174
:102074009DC3217FFCA2401E5F01E3BD3E6082DC64
:10208400237D9FC1421CFEA0E1BF5D0380DE3C6254
:10209400BEE0025CDF81633D7C22C09E1D43A1FF44
:1020A4004618FAA427799BC584DA3866E5BB590734
:1020B400DB856739BAE406581947A5FB7826C49A24
:1020C400653BD987045AB8E6A7F91B45C6987A2414
:1020D400F8A6441A99C7257B3A6486D85B05E7B904
:1020E4008CD2306EEDB3510F4E10F2AC2F7193CDF4
:1020F400114FADF3702ECC92D38D6F31B2EC0E50E4
:10210400AFF1134DCE90722C6D33D18F0C52B0EED3
:10211400326C8ED0530DEFB1F0AE4C1291CF2D73C3
:10212400CA947628ABF517490856B4EA6937D58BB3
:102134005709EBB536688AD495CB2977F4AA4816A3
:10214400E9B7550B88D6346A2B7597C94A14F6A893
:10215400742AC896154BA9F7B6E80A54D7896B3583
:0A21640070B8DCEEF4F7FAFDFEFFA0
:032DD90001640A88
:1025BB00151E151EA81EECF608EDF6151E151E159C
:1025CB001EA81EC6EBC608C6EAC608C6E9C6E51EA7
:0425DB0024FCF51EC9
:1025DF00F80808E4F6A81EF608F6E51E2407F9A881
:1025EF001EE6FE08E6FFC3099719E76480F8EE645C
:1025FF0080985037E51E2404F8CBE6CB08E6FA089E
:10260F00E6F98F828E8312106EA81E080866FFE50A
:10261F001E2403F8EFF6E690206493A81E0808F630
:10262F00A81E0806E61870B20680AFA81E0808E6B6
:01263F00FF9B
:07264000E51E2409F51E222E
:07000300ED6F90206493FFF4
:01000A0022D3
:102D6000EF701E7598D0E589540F4420F58953C83B
:102D7000E1438E10ED90216393F58DD28ED2ACC2DB
:032D8000BCD2AF13
:012D8300222D
:102AB500D2AFD2A9C2BBE589540F4401F589E4F52B
:102AC5008E758CDBF58AD28CF56AF569F568F56744
:102AD500F56EF56DF56CF56B756364FFEF25E02517
:102AE500E024A2F8E4F6EF25E025E024A3F8E4F6D7
:102AF500EF25E025E024A4F8E4F6EF25E025E02421
:082B0500A5F8E4F60FBF01D4AE
:012B0D0022A5
:02251E00151E88
:10252000A81EE4F6A81EE6FFC3940140030225B8E6
:10253000EF25E025E024A5F8E6FFD394004052A85B
:102540001EE625E025E024A3F8E67045EF30E0150F
:10255000A81EE6FF25E025E024A5F8E6D394014077
:10256000047D0080067D01A81EE6FF122C4CA81EEB
:10257000E6FF25E025E024A5F816E66014EF25E047
:1025800025E024A4F8E6FEEF25E025E024A3F8EEFC
:10259000F6A81EE625E025E024A3F8E6600116A8CB
:1025A0001EE6FF25E025E024A5F8E670057D011272
:0825B0002C4CA81E0602252494
:0325B800051E22DB
:03000B0002275376
:10275300C0E0C0F0C083C082C0D0E8C0E0E9C0E000
:10276300EAC0E0EBC0E0ECC0E0EDC0E0EEC0E0EFBB
:10277300C0E0758CDCE56A2401F56AE43569F56926
:10278300E43568F568E43567F567D56318E56E24C5
:1027930001F56EE4356DF56DE4356CF56CE4356B80
:1027A300F56B75636412251E122D84D0E0FFD0E013
:1027B300FED0E0FDD0E0FCD0E0FBD0E0FAD0E0F9C1
:0E27C300D0E0F8D0D0D082D083D0F0D0E03279
:102D3900151EA81EEDF6151EA81EEFF6A81EE6FF25
:102D4900C39401500D08E6FEEF25E025E024A2F822
:072D5900EEF6051E051E2227
:1027D100151E151EA81EEAF608EBF6151EA81EED1D
:1027E100F6151EA81EEFF6A81EE6FFC3940150526F
:1027F100EF25E025E024A5F8E67047A81EE6FB25B5
:10280100E025E024A3F8E67039A81E08E625E004D7
:10281100FFA81EE6FA25E025E024A5F8EFF6A81E9C
:102821000808E6FE08E6FF7C007D0A121136EA255B
:10283100E025E024A4F8EFF6EB25E025E024A3F859
:09284100E4F6E51E2404F51E2254
:102C4C00151EA81EEDF6151EA81EEFF6A81EE6FF13
:102C5C00C39401501CEF25E025E024A2F8E6601196
:102C6C00A81E08E670047F0180027F00A81E08EFF2
:102C7C00F6A81EE6700608E624FF92B4051E051E93
:012C8C002225
:0C2E0E00C2AFAF6AAE69AD68AC67D2AF6E
:012E1A002295
:0C2E1B00C2AFAF6EAE6DAD6CAC6BD2AF51
:012E27002288
:102D1000151EA81EEFF6A81EE67004F565F56630D0
:102D20001014E56475F064A4FFC3E5669FE565953E
:092D3000F0500375FFA5051E22F9
:102DA400D210E4F565F566EF6004F564800375649C
:0E2DB4000A75FF0775FFA543B28075EF09226F
:0E2DF300C210E4F565F56675FFDE75FFAD22D2
:102D84000566E56670020565301014E56475F06447
:102D9400A4FFC3E5669FE56595F0500375FFA52282
:042CE5008E478F483F
:102CE900E4F549F54AC3E54A9548E549954750163B
:102CF9007FE87E03122B0E7F01122D10054AE54A4B
:062D090070E3054980DFC4
:012D0F0022A1
:042B0E008E538F54FF
:102B1200D3E55494FAE5539400500AEFD39400405D
:102B22003C001F80F6855355855456D3E55694FADA
:102B3200E555940040157FFA7E00122B0E7406258F
:102B420056F55674FF3555F55580E0D3E55494009B
:0D2B5200E55394004007AF56AE55122B0E10
:012B5F002253
:10298D007547007548007549417B007A00793F7D98
:01299D000237
:08299E008B438A4489458D46F4
:1029A6007F01122D10AB47AA48A9491211822400B3
:1029B600FFE5F03460FE85434A85444B85454CE48B
:1029C600FDEDC39546501BEF2DF582E43EF583E4FD
:1029D60093AB4AAA4BA94C8D827583001210AD0D9C
:0F29E60080DFAB47AA48A949E48546F00211AD4E
:10231F00754912754A3475510075520075534B7BD0
:07232F00007A0079497D02EC
:082336008B4D8A4E894F8D503A
:10233E007896E664F160030223D5122DF3C2AFE561
:10234E00B654F04408F5B6758F01AB51AA52A95395
:10235E001211822400FFE5F03460789BF608EFF648
:10236E00AA4EA94F789FA64D08C6EAC608C6E9C66A
:10237E00E4789DF6789DE6C395505032789FCBE673
:10238E00CB080806E618CAE6CA70010614F9121040
:10239E0055789EF6E6FF789B0806E618CCE6CC70DC
:1023AE00010614F5828C83EFF0789D0680C6E4F565
:1023BE008F53B6F0AB51AA52A9538550F01211ADFE
:0723CE00D2AFE4FF122DA4C1
:0123D50022E5
:102B60007896E664F1704AC2AF122DF3E5B654F0E0
:102B70004408F5B6758F03789C7660087600E47893
:102B80009BF6789CE6FE08E6F5828E83E4F07F01F2
:102B9000122D10789DE426F618740236F61806E613
:102BA000C3940840DDE4F58F53B6F0D2AFFF122D89
:012BB000A480
:012BB1002201
:10247B00122B60E4F54BF54CF55175520075534B2F
:10248B00FB7A0079087D1612233612231FE4F548D8
:10249B00E548C3781F965073E4F547AB60AA61A972
:1024AB006275F010E547A4F58285F08312106E601B
:1024BB0056E54775F010A429F9EA35F0FA90000DAE
:1024CB001212F17877E68548F0A429F9EA35F0FA8B
:1024DB00EBC0E0EAC0E0E9C0E0AB60AA61A96275BD
:1024EB00F010E547A4F58285F08312106EFD75514F
:1024FB000075520075534BD0E0F9D0E0FAD0E0FBF9
:10250B00122336054780940548808512231FE478F3
:02251B0096F632
:01251D00229B
:10226100E4F541F542F53EF547754800754941FBF6
:102271007A0079087D1612299E12298DE540643471
:102281007004E53F64127003433E01E4F53DE53D12
:10229100C3781F965073E4F53CAB60AA61A96275DF
:1022A100F010E53CA4F58285F08312106E6056E5CE
:1022B1003C75F010A429F9EA35F0FA90000D1212DC
:1022C100F17877E6853DF0A429F9EA35F0FAEBC01B
:1022D100E0EAC0E0E9C0E0AB60AA61A96275F01074
:1022E100E53CA4F58285F08312106EFD75470075FB
:1022F1004800754941D0E0F9D0E0FAD0E0FB12295D
:102301009E053C8094053D808512298DE54064340D
:0D2311007004E53F64127003433E02AF3ECE
:01231E00229C
:100DF000EC4D6011E8497017ED33EC3304600DE4FD
:100E0000FCFFFEFD22E933E8330470F802104012C3
:100E1000100B58046009E4CC2481500628500902C4
:100E2000104A284003021047C0E0EB4A7044B980E2
:100E300006D0E0FB021036EF4E701CBD8008EBFFC1
:100E4000EAFEE9FD80EBE98DF0A4FEE5F0020ED9A3
:100E5000E9CDF9EAFEEBFFEF89F0A4FCE5F0CE89DD
:100E6000F0A42EFFE435F0CD89F0A42DFEE435F09A
:100E70008067EF4E7005BD80D780C3EF8BF0A4ACC8
:100E8000F0EE8BF0A42CFCE435F0F8EF8AF0A42C03
:100E9000E5F038FCE433CB8DF0A42CFCE5F03BF816
:100EA000EE8AF0A42CFCE5F038F8E433CF89F0A406
:100EB0002CFCE5F038CF3400CE89F0A42FFFE5F00C
:100EC0003EFEE433C98DF0A42EFEE5F039CD8AF064
:100ED000A42FFFE5F03EFEE43DFD33D0E0FB5007DC
:100EE0000BBB000F02104AEC2CFCEF33FFEE33FE7D
:060EF000ED33FD021022AB
:100EF60002104AEC5D046005E859047003021040D4
:100F060012100B580460F6EC4860F2EC7004FDFE1B
:100F1600FF22C860DB2481C85009C39860025006CE
:100F26000210479850CAF582E9294B4A7005AB82F0
:100F360002103675F0007C1A7880C3EF9BEE9AEDAE
:100F460099400DC3EF9BFFEE9AFEED99FDE842F046
:100F5600DC23ACF0D0E0FFD0E0FED0E0FDAB822099
:100F6600E7101BEB60BAEC2CFCEF33FFEE33FEED23
:100F760033FD021022E803F830E705C0F075F000F3
:100F8600EF2FFFEE33FEED33FD40B830E7C280AA07
:100F960075F020800E75F010800575F0087D007ED6
:100FA600007F003392D530D5031212B3EC334010D4
:100FB600EF33FFEE33FEED33FDEC33FCD5F0ED22DF
:0E0FC600E5F0247EA2D513CC92E7CDCEFF221B
:100FD400EDD2E7CD33EC3392D524814006E4FFFE15
:100FE400FDFC22FCE4CFCECDCC24E0501174FF8074
:100FF400EDC3CC13CCCD13CDCE13CECF13CF047011
:07100400F030D5DE0212B34B
:10100B00E9D2E7C933E833F892D5EDD2E7CD33EC2B
:07101B0033FC5002B2D522A4
:10102200EC30E7100FBF000C0EBE00080DBD00042F
:101032000BEB6014A2D5EB13FCED92E7FD2274FFDB
:10104200FCFDFEFF22E480F8A2D574FF13FC7D8034
:03105200E480EF48
:030000000226478E
:0C264700787FE4F6D8FD7581A502268E90
:10105500BB010689828A83E0225002E722BBFE0299
:09106500E32289828A83E49322CC
:10106E00BB010CE58229F582E5833AF583E0225037
:10107E0006E92582F8E622BBFE06E92582F8E22281
:0D108E00E58229F582E5833AF583E493229B
:10109B00BB010689828A83F0225002F722BBFE0134
:0210AB00F3222E
:1010AD00F8BB010DE58229F582E5833AF583E8F079
:1010BD00225006E92582C8F622BBFE05E92582C825
:0210CD00F2220D
:1010CF00EF8DF0A4A8F0CF8CF0A428CE8DF0A42E35
:0210DF00FE22EF
:1010E100BC000BBE0029EF8DF084FFADF022E4CCF3
:1010F100F875F008EF2FFFEE33FEEC33FCEE9DECBC
:10110100984005FCEE9DFE0FD5F0E9E4CEFD22ED01
:10111100F8F5F0EE8420D21CFEADF075F008EF2F4B
:10112100FFED33FD4007985006D5F0F222C398FD3C
:051131000FD5F0EA22D9
:10113600C2D5EC30E709B2D5E4C39DFDE49CFCEED4
:1011460030E715B2D5E4C39FFFE49EFE1210E1C35B
:10115600E49DFDE49CFC80031210E130D507C3E456
:061166009FFFE49EFE2243
:10116C00C5F0F8A3E028F0C5F0F8E582158270020E
:06117C001583E038F022AB
:10118200BB010A89828A83E0F5F0A3E02250068738
:10119200F009E71922BBFE07E3F5F009E3192289FA
:0B11A200828A83E493F5F0740193222D
:1011AD00BB010789828A8302116C500B09C5F02798
:1011BD00F7C5F01937F722BBFE0D09F8E325F0F35B
:1011CD00C5F019E338F322F889828A8374019325D7
:0811DD00F0C5F0F8E49338229C
:1011E50075F008758200EF2FFFEE33FECD33CDCCC1
:1011F50033CCC58233C5829BED9AEC99E582984044
:101205000CF582EE9BFEED9AFDEC99FC0FD5F0D620
:10121500E4CEFBE4CDFAE4CCF9A88222B800C1B94A
:101225000059BA002DEC8BF084CFCECDFCE5F0CB88
:10123500F97818EF2FFFEE33FEED33FDEC33FCEBC1
:1012450033FB10D703994004EB99FB0FD8E5E4F97C
:10125500FA227818EF2FFFEE33FEED33FDEC33FC69
:10126500C933C910D7059BE99A4007EC9BFCE99A5D
:10127500F90FD8E0E4C9FAE4CCFB2275F010EF2FA2
:10128500FFEE33FEED33FDCC33CCC833C810D707A2
:101295009BEC9AE899400AED9BFDEC9AFCE899F8DD
:0E12A5000FD5F0DAE4CDFBE4CCFAE4C8F92270
:0E12B300C3E49FFFE49EFEE49DFDE49CFC224C
:1012C100EB9FF5F0EA9E42F0E99D42F0E89C45F083
:0112D10022FA
:1012D200E8600FEFC333FFEE33FEED33FDEC33FC7A
:0312E200D8F1221E
:0C12E500ECF608EDF608EEF608EFF62235
:1012F100BB010DE58229F582E5833AF58302137C72
:101301005007E92582F8021373BBFE07E92582F82D
:10131100021385E58229F582E5833AF58302138E6E
:10132100D083D082F8E4937012740193700DA3A35B
:1013310093F8740193F5828883E47374029368606F
:06134100EFA3A3A380DF6F
:102BB2008B3C8A3D893EE4F544F545E5431543AE39
:102BC20042700215424E6033AB3FAA40A941121037
:102BD20055FFAB3CAA3DA93E0545E545AC44700214
:102BE200054414F5828C83EF1210ADEF60CD7401B1
:102BF2002541F541E43540F54080C0AB3CAA3DA9F2
:022C02003E2270
:10134700EF4E6012EF60010EEDBB010B89828A83BD
:10135700F0A3DFFCDEFA2289F05007F709DFFCA9CA
:0C136700F022BBFEFCF309DFFCA9F02221
:10265300022E28E493A3F8E493A34003F68001F247
:1026630008DFF48029E493A3F85407240CC8C33388
:10267300C4540F4420C8834004F456800146F6DF57
:10268300E4800B0102040810204080902DC2E47EF8
:10269300019360BCA3FF543F30E509541FFEE4934C
:1026A300A360010ECF54C025E060A840B8E493A313
:1026B300FAE493A3F8E493A3C8C582C8CAC583CA3E
:1026C300F0A3C8C582C8CAC583CADFE9DEE780BEF6
:012DDC0000F6
:09137300E6FB08E6FA08E6F9229F
:09137C00E0FBA3E0FAA3E0F92272
:09138500E2FB08E2FA08E2F92299
:0C138E00E493FB740193FA740293F922BB
:00000001FF
